:10740000F201F999FECFF2BDE1BD0895F9DFF89AD6
:1074100080B508C0F5DF1FBA80BD0FB6F894FA9AA0
:10742000F99A0FBE31962F010895E0E0F0E08591C2
:1074300094910196089520E82093610010926100D4
:1074400081E085BF82E085BF81EF85B987EE84B991
:107450001DB8769A10BA80EF81BB84E68BB984EFB1
:107460008AB980E58CBD81E08DBD089580EE8BB931
:107470008BEA37D0109289008AEF8093880082E0EF
:1074800080936F0083E0809381004BD04AD05C985A
:10749000EDE6F7E785913AD0E038E1F781E08093B7
:1074A000D7008AE482BF1092D8001092E2001092B6
:1074B000DA001092E10080E808D019BC1EBA1092E0
:1074C000E0004AD489E03BD481E98093D800089554
:1074D000A3E6B1E090E81AD08D939A95E1F708956C
:1074E00086E008D010C083E005D08F2F0FD08E2FFC
:1074F0000DD080E05E9A5A9809C005D085E0FADF89
:1075000005D080FDFDCF5A9A5E9808958EBD8DB549
:10751000000087FFFCCF8EB508958FE08221E9F748
:10752000F2DFE3E6F6E05C9A40E458E060817181C6
:1075300098E08FEF60FF8F7070FF807FE7DF6695C8
:1075400076959A95B1F7E058FF4F5A9579F7EE5F27
:10755000F3404A9551F70895E3E6F1E097FC36C011
:1075600094FC4DC092FE089526842220E1F3F89405
:10757000C089D78520E030E080E090E4AFEFBFEF36
:10758000119682199040E0F72D01BD4F8D0127FD26
:1075900013C0E0E0F8E011928EE7819392E4E117E6
:1075A00091939AE508F092E4E334C9F7819310824D
:1075B000B7DFFE01219697DF8BDFF901F2D4205867
:1075C0003F4F040D151D2A9411F704C28301282D85
:1075D00060906C0170906B0146D019F48823C1F75C
:1075E0000895380188243FD0E1F580916A0182171F
:1075F00009F4830160906E0170906D01F4CF60908A
:107600006E0170906D012FD081F48823C1F7089529
:107610009FEF95FC08C096FC05C093FE089505DF1A
:10762000E9F3D8C191E097FB890E662477248301A2
:10763000222719D0B1F4882389F380916A0136F0AA
:10764000881650F4821730F0213003C0881520F4DA
:10765000281710F48301282F60906E0170906D013F
:10766000E8CF3801822EF3013EDF32DFC3E6D1E0FE
:10767000E6E6F7E709908591081621F4ED36D1F793
:107680000880801040CFC9E025DFCA95E9F7D0E136
:1076900095FC1EC097FC53C094FC35C0C3E6D2E0F5
:1076A000E3E6F6E098E088E78E0F00840192E817A1
:1076B000E1F7884F09900192E817E1F7C858DF4FCA
:1076C0009A9589F72ADFC85FD340C33E49F749C07E
:1076D000C3E6D6E0EBE5FAE098E08E2F88570290FB
:1076E0000086E817E1F738960A900292E817E1F76A
:1076F0003897C857D0409A9581F70FDFC850DC4FB4
:10770000C33E41F72EC0A3EEB6E0E3E6F6E09AE012
:10771000C6E00D9080818025807F802582958193B1
:10772000A336B90709F4B2E0E336F90709F4F2E049
:10773000E336FC0771F7F1DEDA9529F712C0A3EE04
:10774000B9E0E3E6FAE092E00E90829180258F7036
:10775000802582958083E336F907B1F7DEDEDA957E
:1077600071F78827089541524455424F5915003FFB
:1077700075205FA055A100A200A87F81CFB121AFE5
:107780000000FFFFCFCFFFFFFFFFCFCFFFFF0000C5
:10779000FE067E7E06FE46565616FE0656461EFE21
:1077A0003F61E9E3FFE3EBE3FFE3EBE3FFE16B3F83
:1077B0001201100102000008412336000100000000
:1077C000000109023E0002010080320904000001AC
:1077D000020201000524001001042402040524060D
:1077E0000001070582030800FF09040100020A00E6
:1077F00000000705040210000107058302100001C4
:1078000011241FBE8FEF9AE09EBF8DBF04B714BE38
:1078100088E18093600010926000222433242101CB
:1078200043943101410199C00F928F939F931F920E
:107830000FB60F9211244F936F938091DA0080FF5F
:107840003FC02BC00F920FB68F939F93EF93FF9380
:1078500088278093850080938400E0E5F1E09281A1
:10786000907261F490818917980B908309F45D9A66
:1078700091818917980B918309F4289A239411F424
:107880008315381EFF91EF915CC080E189BD82E1D4
:1078900089BD09B400FEFDCF08958091D80080FF16
:1078A0000FC08091DA008E7F8093DA008091D9003A
:1078B00080FF04C0EADF81E08EBB02C019BC1EBAA3
:1078C0008091E10080FF0BC034D280FF08C034D229
:1078D0008091D8008062F9DD19BC85E08EBB809173
:1078E000E10084FF1AC025D284FF17C0CEDF80914B
:1078F000D8008F7DEADD8FEE2AD01BD28F7E81608B
:107900001ED280915301882331F48091E30087FDDA
:1079100002C081E001C084E08EBB8091E10083FF62
:107920000CC007D283FF09C087EF11D082E08EBB65
:10793000109253010BD000D20FD26F914F910F9044
:107940001F909F918F910FBE0F9018958EEF009012
:10795000E10008220092E10008956DDDA0E0B1E0B1
:10796000E0EBF7E705900D92A035E1F71D92BB30F3
:10797000E9F700FF07C07C9B05C048DD882312F0B3
:1079800054DD41F573DD78946EDE79F0ABE9B7E054
:10799000E0E8F7E703E010E105900D921A95E1F7B2
:1079A000A059BF4F0A95B9F7BCDD51D0EAD28091FA
:1079B0005201807859F48FB18095807F669B8860F2
:1079C0001C9B8460982E24DE8110C6DD33206AF76C
:1079D0002CDD59F3F89489EB84DD81E08093E0009D
:1079E00010926F0010928100109285001092840016
:1079F00081E085BF15BE2E9A2F9A2D9A5D9A289AFE
:107A00000C94000091D107C053D102C0B7D239F015
:107A10008DD182FFFBCF85FFF7CF8091F1000895D4
:107A2000082E83E082D185FD07C077D102C0A6D29F
:107A300069F07CD180FFFBCF0092F1008091520170
:107A4000807221F45D9884E68093500108956CD192
:107A500082FF34C180915201807221F4289884E61B
:107A600080935101CFDF182F853431F422248EE723
:107A7000382EC6DC8DE007C1843511F4C3DFFACFA0
:107A80008C34C1F38035B1F3843721F484E4C8DF4A
:107A900080E0F9C0813611F489E5F5C0813429F41C
:107AA000B1DF582EAFDF482EE5CF803711F483E5E4
:107AB000EAC0833539F4E6E6F7E78591B1DFED36C4
:107AC000E1F7E2C0863521F481E3AADF85E3DBC07C
:107AD000863761F481E3669B8E5F1C9B8F5FA0DF1E
:107AE0008FB1809582958F708F5BCDC08837A9F458
:107AF00089DF80935201289A84FD28985D9A83FD3E
:107B00005D982E9A81FD2E982F9A82FD2F982D9A9E
:107B100080FD2D9887FD8824ADCF8A3649F48FE902
:107B2000E9DCC3E0F3DC7CDFCA95E1F7ECDCACC058
:107B3000833731F487E874DF85E972DF8EE1A3C013
:107B4000853639F4E0E8F3E73FD2E058F040E0F75B
:107B500091CF823631F489E563DF80E061DF80E830
:107B600092C0823419F0873609F079C033244ADF95
:107B7000D82F48DFC82F46DF082F8354843008F001
:107B800081C0063411F4440C551CF20110926F00B0
:107B90001736A1F4033471F483E0A6DCB7DC40DFD0
:107BA0002197E1F7B0DC08C0063411F4859101C0DB
:107BB0002DDC36DF2197C2F72F0149C00334A1F431
:107BC0008E2F8F7021F48CDC80E28EDC96DC88DCDA
:107BD00082E08ADC17DF9ADCCA95E1F78EDC319609
:107BE000DA9571F72F0131C00634F1F49F01F437B3
:107BF000D8F4EAD119C006DF063461F4C0FB46F0C0
:107C0000F43728F4182E81E087BFE89511243296C6
:107C1000082E0AC0043439F4DF01B370AD59B94FEE
:107C20008D93319601C0F6DB21972AF7043431F4A5
:107C30002F01F370FE2B49F474DC07C0063429F4DD
:107C40002F01F901F43708F4BDD18DE0E9DE0634E7
:107C500011F45694479482E080936F0015C08237E8
:107C6000E1E049F08634E0E031F08E34E3E019F0F1
:107C7000813531F4E2E0F0E089E087BF849103C010
:107C80008B3111F08FE3CCDE83E088D146D095FFB5
:107C900003C009C073D191F049D080FFFBCF3DD024
:107CA00002C06CD159F042D080FFFBCF84E076D186
:107CB0008BE734C061D1E4E5F1E067E0089590918D
:107CC0005B0180915C01913231F0913A61F5813232
:107CD00051F5F0DF73C0803231F5ECDF4FD1E9F0C0
:107CE0008530D9F023D083FD18C082FFF7CF04C0C0
:107CF00094DE8193615031F09091F3008091F20015
:107D0000892BB1F7D5DF611549F704C037D129F0C8
:107D1000853019F00BD080FFF9CF8EE79091E80005
:107D200089238093E800089584E038D18091E800A9
:107D300008958091E2000895FCDF8E7F806180933A
:107D4000E200089582E061EC09D083E061E802D0AE
:107D500084E060E842E103C080E060E042E01ED1E0
:107D600081E007D01092ED006093EC004093ED00AD
:107D700008959091EB00892B8093EB00089560E0CB
:107D8000923029F0913031F4E0E062E103C0E2E1A9
:107D90006EE300C0F1E0089580915B0188234CF40C
:107DA00002C0ECD051F0C2DF82FFFBCF81CFE6D022
:107DB00021F0BCDF80FFFBCFB0DF0895409161016F
:107DC000509162014617510510F490E028C06115EA
:107DD00011F0462FFACFA1DF40E0F7CFCFD059F115
:107DE000853049F1A3DF83FD63CFA0DF82FD20C092
:107DF00080FF15C03091F3002091F20005C0819101
:107E00008093F10041502F5F411519F02830310562
:107E1000B0F350E02830310509F451E07EDF411520
:107E2000E9F65523D9F604C0A9D029F0853019F018
:107E30007DDF82FFF9CF3CCFEBE5F1E0EEDD819312
:107E4000E336E1F73CDF72DF83FF91C080915B0195
:107E500090915C01913009F170F09330F1F0953020
:107E600009F444C0963009F456C0983009F460C053
:107E7000993059F767C0823841F780915F018DD002
:107E80002091EB001092E90077D022952695217081
:107E90002093F1001092F10052C0882311F082303B
:107EA000A1F68F71823089F680915D018823D1F42B
:107EB00020915F01277049F22093E9008091EB0047
:107EC00080FF10C0933011F480E20BC080E151DFDD
:107ED00081E0880F2A95E9F78093EA001092EA0082
:107EE00088E047DF1092E90047D02AC0882391F448
:107EF00010915D0110680FB7F8943ED04DDF16DF8A
:107F000080FFFDCF1093E300103883E009F482E096
:107F10008EBB0FBF2CC08058823048F580915D0128
:107F200090915E012CDF603011F126D047DF1FC039
:107F30008038E9F421D0809153018093F100EDDE87
:107F40002BDF15C0882399F490915D01923078F46D
:107F50009093530111D020DF80915301882321F4A5
:107F60008091E30091E087FD94E09EBBEBDEDEDED6
:107F700083FF089580E2FDDE87EFD0CE8EB38823A5
:107F80000895FCDF69F08091E9008F931092E90079
:107F9000CDDE83FF01C050DF8F9187708093E900B1
:107FA0000895A3E6B1E0F437B8F40ED090E40D9054
:107FB0001D9081E087BFE89532969A95C1F711240C
:107FC000E058F04085E001C083E001D081E187BF47
:0A7FD000E89507B600FCFDCF089508
:047FFC00D4CFFBDC07
:040000030000740085
:00000001FF
